:1000000000308A007F2800000000253084000008AE
:10001000031918280130A100A001A00B0D28A10B85
:100020000C284830A000A00B13280000800B0A28E1
:1000300000340830A1008316051283120516A1179B
:100040002E28A113A70C03180512031C051621174F
:100050002E282113A10B222805122E281E308400E1
:10006000840B3028A11B2128211B292800342808B3
:10007000A101270203183F282708A0004B28A00150
:100080000830A900A70DA00D280820020318A00021
:10009000A10DA90B4228003426186628A618792835
:1000A0002508A7006430A80037202008A5002108F3
:1000B0003030031D602826196628A61920306228D2
:1000C0002611A611A1072108A70019202508A700BD
:1000D0000A30A80037202008A50021083030031D71
:1000E000752826197928A6192030A1072108A7000C
:1000F00019203030A5072508A700192000348401F5
:1001000083019F308400073080008316051283121C
:1001100005161F083839C1389F000030A1001F089C
:10012000C73921049F00A4010830A1001F08C73966
:1001300021049F000230A50005201F151F199E28CD
:100140001E08A2001030A1001F08C73921049F001B
:100150000230A50005201F151F19AC281E08A3009A
:100160002530A70019202208A500A6014C202C301C
:10017000A70019202308A500A6014C200D30A700D8
:1001800019200A30A7001920A408031DCE28013029
:10019000A4008316851183128515D328A401831624
:0A01A0008511831285119428630075
:02400E00F43F7D
:0207FE0088343D
:00000001FF
